 mexit01

 Timestamp is ee0aed6c (reproducible build file hash)

 Preferred load address is 0000000180000000

 Start         Length     Name                   Class
 0001:00000000 00001c50H .text$mn                CODE
 0001:00001c50 00000036H .text$mn$00             CODE
 0001:00001c86 00000092H .text$x                 CODE
 0002:00000000 00000160H .idata$5                DATA
 0002:00000160 00000038H .00cfg                  DATA
 0002:00000198 00000008H .CRT$XCA                DATA
 0002:000001a0 00000008H .CRT$XCZ                DATA
 0002:000001a8 00000008H .CRT$XIA                DATA
 0002:000001b0 00000008H .CRT$XIC                DATA
 0002:000001b8 00000008H .CRT$XIZ                DATA
 0002:000001c0 00000008H .CRT$XLA                DATA
 0002:000001c8 00000008H .CRT$XLZ                DATA
 0002:000001d0 00000008H .CRT$XPA                DATA
 0002:000001d8 00000008H .CRT$XPZ                DATA
 0002:000001e0 00000008H .CRT$XTA                DATA
 0002:000001e8 00000008H .CRT$XTZ                DATA
 0002:000001f0 00000000H .gehcont$y              DATA
 0002:000001f0 00000000H .gfids$y                DATA
 0002:000001f0 00000e90H .rdata                  DATA
 0002:00001080 00000000H .rdata$CastGuardVftablesA DATA
 0002:00001080 00000000H .rdata$CastGuardVftablesC DATA
 0002:00001080 00000028H .rdata$T                DATA
 0002:000010a8 00000064H .rdata$voltmd           DATA
 0002:0000110c 00000314H .rdata$zzzdbg           DATA
 0002:00001420 00000008H .rtc$IAA                DATA
 0002:00001428 00000008H .rtc$IZZ                DATA
 0002:00001430 00000008H .rtc$TAA                DATA
 0002:00001438 00000008H .rtc$TZZ                DATA
 0002:00001440 00000004H .tls                    DATA
 0002:00001444 00000004H .tls$                   DATA
 0002:00001448 00000008H .tls$ZZZ                DATA
 0002:00001450 000001f0H .xdata                  DATA
 0002:00001640 000000bcH .edata                  DATA
 0002:000016fc 00000064H .idata$2                DATA
 0002:00001760 00000018H .idata$3                DATA
 0002:00001778 00000160H .idata$4                DATA
 0002:000018d8 000003caH .idata$6                DATA
 0003:00000000 00000090H .data                   DATA
 0003:00000090 000007a8H .bss                    DATA
 0004:00000000 00000258H .pdata                  DATA

  Address         Publics by Value              Rva+Base               Lib:Object

 0000:00000000       __AbsoluteZero             0000000000000000     <absolute>
 0000:00000000       ___safe_se_handler_count   0000000000000000     <absolute>
 0000:00000000       ___safe_se_handler_table   0000000000000000     <absolute>
 0000:00000000       __arm64x_extra_rfe_table   0000000000000000     <absolute>
 0000:00000000       __arm64x_extra_rfe_table_size 0000000000000000     <absolute>
 0000:00000000       __arm64x_native_entrypoint 0000000000000000     <absolute>
 0000:00000000       __arm64x_redirection_metadata 0000000000000000     <absolute>
 0000:00000000       __arm64x_redirection_metadata_count 0000000000000000     <absolute>
 0000:00000000       __dynamic_value_reloc_table 0000000000000000     <absolute>
 0000:00000000       __enclave_config           0000000000000000     <absolute>
 0000:00000000       __guard_check_icall_a64n_fptr 0000000000000000     <absolute>
 0000:00000000       __guard_eh_cont_count      0000000000000000     <absolute>
 0000:00000000       __guard_eh_cont_table      0000000000000000     <absolute>
 0000:00000000       __guard_fids_count         0000000000000000     <absolute>
 0000:00000000       __guard_fids_table         0000000000000000     <absolute>
 0000:00000000       __guard_iat_count          0000000000000000     <absolute>
 0000:00000000       __guard_iat_table          0000000000000000     <absolute>
 0000:00000000       __guard_longjmp_count      0000000000000000     <absolute>
 0000:00000000       __guard_longjmp_table      0000000000000000     <absolute>
 0000:00000000       __hybrid_auxiliary_iat     0000000000000000     <absolute>
 0000:00000000       __hybrid_auxiliary_iat_copy 0000000000000000     <absolute>
 0000:00000000       __hybrid_code_map          0000000000000000     <absolute>
 0000:00000000       __hybrid_code_map_count    0000000000000000     <absolute>
 0000:00000000       __x64_code_ranges_to_entry_points 0000000000000000     <absolute>
 0000:00000000       __x64_code_ranges_to_entry_points_count 0000000000000000     <absolute>
 0000:00000100       __guard_flags              0000000000000100     <absolute>
 0000:00000000       __ImageBase                0000000180000000     <linker-defined>
 0001:00000000       ?CallStaticVoidMethod@JNIEnv_@@QEAAXPEAV_jclass@@PEAU_jmethodID@@ZZ 0000000180001000 f i libmexit01.obj
 0001:00000024       ?SetEventNotificationMode@_jvmtiEnv@@QEAA?AW4jvmtiError@@W4jvmtiEventMode@@W4jvmtiEvent@@PEAV_jobject@@ZZ 0000000180001024 f i libmexit01.obj
 0001:00000030       ?TranslateError@@YAPEBDW4jvmtiError@@@Z 0000000180001030 f   libmexit01.obj
 0001:000002e8       ?jlong_to_string@@YAPEAD_JPEAD@Z 00000001800012e8 f   libmexit01.obj
 0001:00000390       Agent_Initialize           0000000180001390 f   libmexit01.obj
 0001:00000514       Agent_OnAttach             0000000180001514 f   libmexit01.obj
 0001:00000514       Agent_OnLoad               0000000180001514 f   libmexit01.obj
 0001:0000051c       Java_mexit01_check         000000018000151c f   libmexit01.obj
 0001:000006d8       Java_mexit01_init0         00000001800016d8 f   libmexit01.obj
 0001:0000077c       Java_mexit01a_chain        000000018000177c f   libmexit01.obj
 0001:000007a8       MethodExit                 00000001800017a8 f   libmexit01.obj
 0001:00000ccc       __local_stdio_printf_options 0000000180001ccc f i libmexit01.obj
 0001:00000cd4       printf                     0000000180001cd4 f i libmexit01.obj
 0001:00000e1c       __GSHandlerCheck           0000000180001e1c f   MSVCRT:gshandler.obj
 0001:00000e3c       __GSHandlerCheckCommon     0000000180001e3c f   MSVCRT:gshandler.obj
 0001:00000eb0       __security_check_cookie    0000000180001eb0 f   MSVCRT:amdsecgs.obj
 0001:000011f0       _DllMainCRTStartup         00000001800021f0 f   MSVCRT:dll_dllmain.obj
 0001:00001230       __scrt_acquire_startup_lock 0000000180002230 f   MSVCRT:utility.obj
 0001:0000126c       __scrt_dllmain_after_initialize_c 000000018000226c f   MSVCRT:utility.obj
 0001:000012a0       __scrt_dllmain_before_initialize_c 00000001800022a0 f   MSVCRT:utility.obj
 0001:000012b8       __scrt_dllmain_crt_thread_attach 00000001800022b8 f   MSVCRT:utility.obj
 0001:000012e0       __scrt_dllmain_crt_thread_detach 00000001800022e0 f   MSVCRT:utility.obj
 0001:000012f8       __scrt_dllmain_exception_filter 00000001800022f8 f   MSVCRT:utility.obj
 0001:00001358       __scrt_dllmain_uninitialize_c 0000000180002358 f   MSVCRT:utility.obj
 0001:00001388       __scrt_dllmain_uninitialize_critical 0000000180002388 f   MSVCRT:utility.obj
 0001:0000139c       __scrt_initialize_crt      000000018000239c f   MSVCRT:utility.obj
 0001:000013e8       __scrt_initialize_onexit_tables 00000001800023e8 f   MSVCRT:utility.obj
 0001:00001474       __scrt_is_nonwritable_in_current_image 0000000180002474 f   MSVCRT:utility.obj
 0001:0000150c       __scrt_release_startup_lock 000000018000250c f   MSVCRT:utility.obj
 0001:00001530       __scrt_uninitialize_crt    0000000180002530 f   MSVCRT:utility.obj
 0001:0000155c       _onexit                    000000018000255c f   MSVCRT:utility.obj
 0001:00001598       atexit                     0000000180002598 f   MSVCRT:utility.obj
 0001:000015b0       __crt_debugger_hook        00000001800025b0 f   MSVCRT:utility_desktop.obj
 0001:000015b8       __scrt_fastfail            00000001800025b8 f   MSVCRT:utility_desktop.obj
 0001:00001704       _guard_check_icall_nop     0000000180002704 f i MSVCRT:guard_support.obj
 0001:00001708       __raise_securityfailure    0000000180002708 f   MSVCRT:gs_report.obj
 0001:0000173c       __report_gsfailure         000000018000273c f   MSVCRT:gs_report.obj
 0001:00001884       __security_init_cookie     0000000180002884 f   MSVCRT:gs_support.obj
 0001:00001930       DllMain                    0000000180002930 f   MSVCRT:dll_dllmain_stub.obj
 0001:00001954       ?__scrt_initialize_type_info@@YAXXZ 0000000180002954 f   MSVCRT:tncleanup.obj
 0001:00001964       ?__scrt_uninitialize_type_info@@YAXXZ 0000000180002964 f   MSVCRT:tncleanup.obj
 0001:00001970       __local_stdio_scanf_options 0000000180002970 f i MSVCRT:default_local_stdio_options.obj
 0001:00001978       __scrt_initialize_default_local_stdio_options 0000000180002978 f   MSVCRT:default_local_stdio_options.obj
 0001:00001994       __scrt_get_dyn_tls_init_callback 0000000180002994 f   MSVCRT:dyn_tls_init.obj
 0001:0000199c       _RTC_Initialize            000000018000299c f   MSVCRT:initsect.obj
 0001:000019d8       _RTC_Terminate             00000001800029d8 f   MSVCRT:initsect.obj
 0001:00001a14       __isa_available_init       0000000180002a14 f   MSVCRT:cpu_disp.obj
 0001:00001bc0       _get_startup_argv_mode     0000000180002bc0 f   MSVCRT:argv_mode.obj
 0001:00001bc8       __scrt_is_ucrt_dll_in_use  0000000180002bc8 f   MSVCRT:ucrt_detection.obj
 0001:00001be0       __C_specific_handler       0000000180002be0 f   vcruntime:VCRUNTIME140.dll
 0001:00001be6       memset                     0000000180002be6 f   vcruntime:VCRUNTIME140.dll
 0001:00001bec       __std_type_info_destroy_list 0000000180002bec f   vcruntime:VCRUNTIME140.dll
 0001:00001bf2       strcmp                     0000000180002bf2 f   ucrt:api-ms-win-crt-string-l1-1-0.dll
 0001:00001bf8       _initterm                  0000000180002bf8 f   ucrt:api-ms-win-crt-runtime-l1-1-0.dll
 0001:00001bfe       _initterm_e                0000000180002bfe f   ucrt:api-ms-win-crt-runtime-l1-1-0.dll
 0001:00001c04       _seh_filter_dll            0000000180002c04 f   ucrt:api-ms-win-crt-runtime-l1-1-0.dll
 0001:00001c0a       _configure_narrow_argv     0000000180002c0a f   ucrt:api-ms-win-crt-runtime-l1-1-0.dll
 0001:00001c10       _initialize_narrow_environment 0000000180002c10 f   ucrt:api-ms-win-crt-runtime-l1-1-0.dll
 0001:00001c16       _initialize_onexit_table   0000000180002c16 f   ucrt:api-ms-win-crt-runtime-l1-1-0.dll
 0001:00001c1c       _register_onexit_function  0000000180002c1c f   ucrt:api-ms-win-crt-runtime-l1-1-0.dll
 0001:00001c22       _execute_onexit_table      0000000180002c22 f   ucrt:api-ms-win-crt-runtime-l1-1-0.dll
 0001:00001c28       _crt_atexit                0000000180002c28 f   ucrt:api-ms-win-crt-runtime-l1-1-0.dll
 0001:00001c2e       _cexit                     0000000180002c2e f   ucrt:api-ms-win-crt-runtime-l1-1-0.dll
 0001:00001c34       __acrt_initialize          0000000180002c34 f   MSVCRT:ucrt_stubs.obj
 0001:00001c34       __acrt_thread_attach       0000000180002c34 f   MSVCRT:ucrt_stubs.obj
 0001:00001c34       __acrt_thread_detach       0000000180002c34 f   MSVCRT:ucrt_stubs.obj
 0001:00001c34       __acrt_uninitialize        0000000180002c34 f   MSVCRT:ucrt_stubs.obj
 0001:00001c34       __acrt_uninitialize_critical 0000000180002c34 f   MSVCRT:ucrt_stubs.obj
 0001:00001c34       __scrt_stub_for_acrt_initialize 0000000180002c34 f   MSVCRT:ucrt_stubs.obj
 0001:00001c34       __scrt_stub_for_acrt_thread_attach 0000000180002c34 f   MSVCRT:ucrt_stubs.obj
 0001:00001c34       __scrt_stub_for_acrt_thread_detach 0000000180002c34 f   MSVCRT:ucrt_stubs.obj
 0001:00001c34       __scrt_stub_for_acrt_uninitialize 0000000180002c34 f   MSVCRT:ucrt_stubs.obj
 0001:00001c34       __scrt_stub_for_acrt_uninitialize_critical 0000000180002c34 f   MSVCRT:ucrt_stubs.obj
 0001:00001c34       __vcrt_initialize          0000000180002c34 f   MSVCRT:ucrt_stubs.obj
 0001:00001c34       __vcrt_thread_attach       0000000180002c34 f   MSVCRT:ucrt_stubs.obj
 0001:00001c34       __vcrt_thread_detach       0000000180002c34 f   MSVCRT:ucrt_stubs.obj
 0001:00001c34       __vcrt_uninitialize        0000000180002c34 f   MSVCRT:ucrt_stubs.obj
 0001:00001c34       __vcrt_uninitialize_critical 0000000180002c34 f   MSVCRT:ucrt_stubs.obj
 0001:00001c38       __scrt_stub_for_is_c_termination_complete 0000000180002c38 f   MSVCRT:ucrt_stubs.obj
 0001:00001c38       _is_c_termination_complete 0000000180002c38 f   MSVCRT:ucrt_stubs.obj
 0001:00001c3b       memcpy                     0000000180002c3b f   vcruntime:VCRUNTIME140.dll
 0001:00001c60       _guard_dispatch_icall_nop  0000000180002c60 f   MSVCRT:guard_dispatch.obj
 0001:00001c80       _guard_xfg_dispatch_icall_nop 0000000180002c80 f   MSVCRT:guard_xfg_dispatch.obj
 0002:00000000       __imp_CloseHandle          0000000180003000     kernel32:KERNEL32.dll
 0002:00000008       __imp_InitializeCriticalSectionAndSpinCount 0000000180003008     kernel32:KERNEL32.dll
 0002:00000010       __imp_DeleteCriticalSection 0000000180003010     kernel32:KERNEL32.dll
 0002:00000018       __imp_CreateEventW         0000000180003018     kernel32:KERNEL32.dll
 0002:00000020       __imp_GetModuleHandleW     0000000180003020     kernel32:KERNEL32.dll
 0002:00000028       __imp_GetProcAddress       0000000180003028     kernel32:KERNEL32.dll
 0002:00000030       __imp_RtlCaptureContext    0000000180003030     kernel32:KERNEL32.dll
 0002:00000038       __imp_RtlLookupFunctionEntry 0000000180003038     kernel32:KERNEL32.dll
 0002:00000040       __imp_RtlVirtualUnwind     0000000180003040     kernel32:KERNEL32.dll
 0002:00000048       __imp_IsDebuggerPresent    0000000180003048     kernel32:KERNEL32.dll
 0002:00000050       __imp_UnhandledExceptionFilter 0000000180003050     kernel32:KERNEL32.dll
 0002:00000058       __imp_SetUnhandledExceptionFilter 0000000180003058     kernel32:KERNEL32.dll
 0002:00000060       __imp_IsProcessorFeaturePresent 0000000180003060     kernel32:KERNEL32.dll
 0002:00000068       __imp_GetCurrentProcess    0000000180003068     kernel32:KERNEL32.dll
 0002:00000070       __imp_TerminateProcess     0000000180003070     kernel32:KERNEL32.dll
 0002:00000078       __imp_QueryPerformanceCounter 0000000180003078     kernel32:KERNEL32.dll
 0002:00000080       __imp_GetCurrentProcessId  0000000180003080     kernel32:KERNEL32.dll
 0002:00000088       __imp_GetCurrentThreadId   0000000180003088     kernel32:KERNEL32.dll
 0002:00000090       __imp_GetSystemTimeAsFileTime 0000000180003090     kernel32:KERNEL32.dll
 0002:00000098       __imp_DisableThreadLibraryCalls 0000000180003098     kernel32:KERNEL32.dll
 0002:000000a0       __imp_InitializeSListHead  00000001800030a0     kernel32:KERNEL32.dll
 0002:000000a8       \177KERNEL32_NULL_THUNK_DATA 00000001800030a8     kernel32:KERNEL32.dll
 0002:000000b0       __imp___C_specific_handler 00000001800030b0     vcruntime:VCRUNTIME140.dll
 0002:000000b8       __imp_memset               00000001800030b8     vcruntime:VCRUNTIME140.dll
 0002:000000c0       __imp___std_type_info_destroy_list 00000001800030c0     vcruntime:VCRUNTIME140.dll
 0002:000000c8       __imp_memcpy               00000001800030c8     vcruntime:VCRUNTIME140.dll
 0002:000000d0       \177VCRUNTIME140_NULL_THUNK_DATA 00000001800030d0     vcruntime:VCRUNTIME140.dll
 0002:000000d8       __imp__initialize_onexit_table 00000001800030d8     ucrt:api-ms-win-crt-runtime-l1-1-0.dll
 0002:000000e0       __imp__cexit               00000001800030e0     ucrt:api-ms-win-crt-runtime-l1-1-0.dll
 0002:000000e8       __imp__crt_atexit          00000001800030e8     ucrt:api-ms-win-crt-runtime-l1-1-0.dll
 0002:000000f0       __imp__execute_onexit_table 00000001800030f0     ucrt:api-ms-win-crt-runtime-l1-1-0.dll
 0002:000000f8       __imp__initterm            00000001800030f8     ucrt:api-ms-win-crt-runtime-l1-1-0.dll
 0002:00000100       __imp__initterm_e          0000000180003100     ucrt:api-ms-win-crt-runtime-l1-1-0.dll
 0002:00000108       __imp__seh_filter_dll      0000000180003108     ucrt:api-ms-win-crt-runtime-l1-1-0.dll
 0002:00000110       __imp__configure_narrow_argv 0000000180003110     ucrt:api-ms-win-crt-runtime-l1-1-0.dll
 0002:00000118       __imp__register_onexit_function 0000000180003118     ucrt:api-ms-win-crt-runtime-l1-1-0.dll
 0002:00000120       __imp__initialize_narrow_environment 0000000180003120     ucrt:api-ms-win-crt-runtime-l1-1-0.dll
 0002:00000128       \177api-ms-win-crt-runtime-l1-1-0_NULL_THUNK_DATA 0000000180003128     ucrt:api-ms-win-crt-runtime-l1-1-0.dll
 0002:00000130       __imp___acrt_iob_func      0000000180003130     ucrt:api-ms-win-crt-stdio-l1-1-0.dll
 0002:00000138       __imp___stdio_common_vfprintf 0000000180003138     ucrt:api-ms-win-crt-stdio-l1-1-0.dll
 0002:00000140       __imp_fflush               0000000180003140     ucrt:api-ms-win-crt-stdio-l1-1-0.dll
 0002:00000148       \177api-ms-win-crt-stdio-l1-1-0_NULL_THUNK_DATA 0000000180003148     ucrt:api-ms-win-crt-stdio-l1-1-0.dll
 0002:00000150       __imp_strcmp               0000000180003150     ucrt:api-ms-win-crt-string-l1-1-0.dll
 0002:00000158       \177api-ms-win-crt-string-l1-1-0_NULL_THUNK_DATA 0000000180003158     ucrt:api-ms-win-crt-string-l1-1-0.dll
 0002:00000160       __guard_check_icall_fptr   0000000180003160     MSVCRT:guard_support.obj
 0002:00000168       __guard_xfg_check_icall_fptr 0000000180003168     MSVCRT:guard_support.obj
 0002:00000170       __guard_dispatch_icall_fptr 0000000180003170     MSVCRT:guard_support.obj
 0002:00000178       __guard_xfg_dispatch_icall_fptr 0000000180003178     MSVCRT:guard_support.obj
 0002:00000180       __guard_xfg_table_dispatch_icall_fptr 0000000180003180     MSVCRT:guard_support.obj
 0002:00000188       __castguard_check_failure_os_handled_fptr 0000000180003188     MSVCRT:guard_support.obj
 0002:00000190       __guard_memcpy_fptr        0000000180003190     vcruntime:softmemtag.obj
 0002:00000198       __xc_a                     0000000180003198     MSVCRT:initializers.obj
 0002:000001a0       __xc_z                     00000001800031a0     MSVCRT:initializers.obj
 0002:000001a8       __xi_a                     00000001800031a8     MSVCRT:initializers.obj
 0002:000001b8       __xi_z                     00000001800031b8     MSVCRT:initializers.obj
 0002:000001c0       __xl_a                     00000001800031c0     MSVCRT:tlssup.obj
 0002:000001c8       __xl_z                     00000001800031c8     MSVCRT:tlssup.obj
 0002:000001d0       __xp_a                     00000001800031d0     MSVCRT:initializers.obj
 0002:000001d8       __xp_z                     00000001800031d8     MSVCRT:initializers.obj
 0002:000001e0       __xt_a                     00000001800031e0     MSVCRT:initializers.obj
 0002:000001e8       __xt_z                     00000001800031e8     MSVCRT:initializers.obj
 0002:000001f0       ??_C@_0L@BHPOCLLJ@Lmexit01a?$DL@ 00000001800031f0     libmexit01.obj
 0002:000001fc       ??_C@_05FGPNDJME@chain@    00000001800031fc     libmexit01.obj
 0002:00000204       ??_C@_03GAEACAIP@?$CI?$CJV@ 0000000180003204     libmexit01.obj
 0002:00000208       ??_C@_05JLNEMJLN@dummy@    0000000180003208     libmexit01.obj
 0002:00000210       ??_C@_0BB@JCNMKLLK@JVMTI_ERROR_NONE@ 0000000180003210     libmexit01.obj
 0002:00000228       ??_C@_0BL@LDIMKLPH@JVMTI_ERROR_INVALID_THREAD@ 0000000180003228     libmexit01.obj
 0002:00000248       ??_C@_0CB@PJFPAIKJ@JVMTI_ERROR_INVALID_THREAD_GROU@ 0000000180003248     libmexit01.obj
 0002:00000270       ??_C@_0BN@LLMKHMNF@JVMTI_ERROR_INVALID_PRIORITY@ 0000000180003270     libmexit01.obj
 0002:00000290       ??_C@_0CB@MBOFKAGB@JVMTI_ERROR_THREAD_NOT_SUSPENDE@ 0000000180003290     libmexit01.obj
 0002:000002b8       ??_C@_0BN@FABOLPBI@JVMTI_ERROR_THREAD_SUSPENDED@ 00000001800032b8     libmexit01.obj
 0002:000002d8       ??_C@_0BN@FDGNOBJM@JVMTI_ERROR_THREAD_NOT_ALIVE@ 00000001800032d8     libmexit01.obj
 0002:000002f8       ??_C@_0BL@GOBIFKNJ@JVMTI_ERROR_INVALID_OBJECT@ 00000001800032f8     libmexit01.obj
 0002:00000318       ??_C@_0BK@FCMAJPPC@JVMTI_ERROR_INVALID_CLASS@ 0000000180003318     libmexit01.obj
 0002:00000338       ??_C@_0BP@IKLLBKEB@JVMTI_ERROR_CLASS_NOT_PREPARED@ 0000000180003338     libmexit01.obj
 0002:00000358       ??_C@_0BN@KLPPLKG@JVMTI_ERROR_INVALID_METHODID@ 0000000180003358     libmexit01.obj
 0002:00000378       ??_C@_0BN@BCEKOKND@JVMTI_ERROR_INVALID_LOCATION@ 0000000180003378     libmexit01.obj
 0002:00000398       ??_C@_0BM@DFDGPME@JVMTI_ERROR_INVALID_FIELDID@ 0000000180003398     libmexit01.obj
 0002:000003b8       ??_C@_0BL@NELIEPEC@JVMTI_ERROR_NO_MORE_FRAMES@ 00000001800033b8     libmexit01.obj
 0002:000003d8       ??_C@_0BJ@BDBECFDM@JVMTI_ERROR_OPAQUE_FRAME@ 00000001800033d8     libmexit01.obj
 0002:000003f8       ??_C@_0BK@MIIFNLOB@JVMTI_ERROR_TYPE_MISMATCH@ 00000001800033f8     libmexit01.obj
 0002:00000418       ??_C@_0BJ@HPCAOILC@JVMTI_ERROR_INVALID_SLOT@ 0000000180003418     libmexit01.obj
 0002:00000438       ??_C@_0BG@CHILOPNI@JVMTI_ERROR_DUPLICATE@ 0000000180003438     libmexit01.obj
 0002:00000450       ??_C@_0BG@DIEMLHKM@JVMTI_ERROR_NOT_FOUND@ 0000000180003450     libmexit01.obj
 0002:00000468       ??_C@_0BM@NHMCKHOB@JVMTI_ERROR_INVALID_MONITOR@ 0000000180003468     libmexit01.obj
 0002:00000488       ??_C@_0BO@PPEDAJGL@JVMTI_ERROR_NOT_MONITOR_OWNER@ 0000000180003488     libmexit01.obj
 0002:000004a8       ??_C@_0BG@FCAIPEID@JVMTI_ERROR_INTERRUPT@ 00000001800034a8     libmexit01.obj
 0002:000004c0       ??_C@_0CB@EGDBNKOI@JVMTI_ERROR_INVALID_CLASS_FORMA@ 00000001800034c0     libmexit01.obj
 0002:000004e8       ??_C@_0CG@DGKOGIAL@JVMTI_ERROR_CIRCULAR_CLASS_DEFI@ 00000001800034e8     libmexit01.obj
 0002:00000510       ??_C@_0BP@ICEALPKC@JVMTI_ERROR_FAILS_VERIFICATION@ 0000000180003510     libmexit01.obj
 0002:00000530       ??_C@_0DC@JDACLMIO@JVMTI_ERROR_UNSUPPORTED_REDEFIN@ 0000000180003530     libmexit01.obj
 0002:00000568       ??_C@_0DE@GKDKNOMJ@JVMTI_ERROR_UNSUPPORTED_REDEFIN@ 0000000180003568     libmexit01.obj
 0002:000005a0       ??_C@_0BO@LAFKIOG@JVMTI_ERROR_INVALID_TYPESTATE@ 00000001800035a0     libmexit01.obj
 0002:000005c0       ??_C@_0DH@INDGCLLB@JVMTI_ERROR_UNSUPPORTED_REDEFIN@ 00000001800035c0     libmexit01.obj
 0002:000005f8       ??_C@_0DE@NHEOMMGI@JVMTI_ERROR_UNSUPPORTED_REDEFIN@ 00000001800035f8     libmexit01.obj
 0002:00000630       ??_C@_0CA@EKPNJOEP@JVMTI_ERROR_UNSUPPORTED_VERSION@ 0000000180003630     libmexit01.obj
 0002:00000650       ??_C@_0BN@OFFMAHHL@JVMTI_ERROR_NAMES_DONT_MATCH@ 0000000180003650     libmexit01.obj
 0002:00000670       ??_C@_0DN@HHBBLAKE@JVMTI_ERROR_UNSUPPORTED_REDEFIN@ 0000000180003670     libmexit01.obj
 0002:000006b0       ??_C@_0DO@HMBGBGNA@JVMTI_ERROR_UNSUPPORTED_REDEFIN@ 00000001800036b0     libmexit01.obj
 0002:000006f0       ??_C@_0BP@PBECGKHJ@JVMTI_ERROR_UNMODIFIABLE_CLASS@ 00000001800036f0     libmexit01.obj
 0002:00000710       ??_C@_0BK@CANILEHF@JVMTI_ERROR_NOT_AVAILABLE@ 0000000180003710     libmexit01.obj
 0002:00000730       ??_C@_0CE@INJKMEFK@JVMTI_ERROR_MUST_POSSESS_CAPABI@ 0000000180003730     libmexit01.obj
 0002:00000758       ??_C@_0BJ@LBFPFPDM@JVMTI_ERROR_NULL_POINTER@ 0000000180003758     libmexit01.obj
 0002:00000778       ??_C@_0BP@CHJPNNEM@JVMTI_ERROR_ABSENT_INFORMATION@ 0000000180003778     libmexit01.obj
 0002:00000798       ??_C@_0BP@OMFMNLC@JVMTI_ERROR_INVALID_EVENT_TYPE@ 0000000180003798     libmexit01.obj
 0002:000007b8       ??_C@_0BN@BIBNPHHO@JVMTI_ERROR_ILLEGAL_ARGUMENT@ 00000001800037b8     libmexit01.obj
 0002:000007d8       ??_C@_0BK@KKNDHDCE@JVMTI_ERROR_NATIVE_METHOD@ 00000001800037d8     libmexit01.obj
 0002:000007f8       ??_C@_0BK@PMKCFHAE@JVMTI_ERROR_OUT_OF_MEMORY@ 00000001800037f8     libmexit01.obj
 0002:00000818       ??_C@_0BK@NNJBDMNB@JVMTI_ERROR_ACCESS_DENIED@ 0000000180003818     libmexit01.obj
 0002:00000838       ??_C@_0BI@GHECLMNC@JVMTI_ERROR_WRONG_PHASE@ 0000000180003838     libmexit01.obj
 0002:00000850       ??_C@_0BF@OLIHJOII@JVMTI_ERROR_INTERNAL@ 0000000180003850     libmexit01.obj
 0002:00000868       ??_C@_0BO@EOHGKJHI@JVMTI_ERROR_UNATTACHED_THREAD@ 0000000180003868     libmexit01.obj
 0002:00000888       ??_C@_0CA@LKHFDACL@JVMTI_ERROR_INVALID_ENVIRONMENT@ 0000000180003888     libmexit01.obj
 0002:000008a8       ??_C@_0BA@MMFHLOKK@?$DMunknown?5error?$DO@ 00000001800038a8     libmexit01.obj
 0002:000008b8       ??_C@_0DF@BMPOKPHD@?$CIGetMethodDeclaringClass?$CJ?5unexp@ 00000001800038b8     libmexit01.obj
 0002:000008f0       ??_C@_0CP@HMGAFMHE@?$CIGetClassSignature?$CJ?5unexpected?5@ 00000001800038f0     libmexit01.obj
 0002:00000920       ??_C@_0CF@KMFEIAOJ@?$DO?$DO?$DO?5retrieving?5method?5exit?5info@ 0000000180003920     libmexit01.obj
 0002:00000948       ??_C@_0CL@MEMLFJHD@?$CIGetMethodName?$CJ?5unexpected?5erro@ 0000000180003948     libmexit01.obj
 0002:00000978       ??_C@_0CO@HJKAMPK@?$CIGetFrameLocation?$CJ?5unexpected?5e@ 0000000180003978     libmexit01.obj
 0002:000009a8       ??_C@_0BG@KNOALIEJ@?$DO?$DO?$DO?5?5?5?5?5?5class?3?5?$CC?$CFs?$CC?6@ 00000001800039a8     libmexit01.obj
 0002:000009c0       ??_C@_0BI@NIFPBCMG@?$DO?$DO?$DO?5?5?5?5?5method?3?5?$CC?$CFs?$CFs?$CC?6@ 00000001800039c0     libmexit01.obj
 0002:000009d8       ??_C@_0BE@KKELBFJG@?$DO?$DO?$DO?5?5?5location?3?5?$CFs?6@ 00000001800039d8     libmexit01.obj
 0002:000009f0       ??_C@_0O@BHPJPDFF@?$DO?$DO?$DO?5?4?4?4?5done?6@ 00000001800039f0     libmexit01.obj
 0002:00000a00       ??_C@_0BO@IPCBIMP@?$CIexit?$CD?$CFllu?$CJ?5wrong?5class?3?5?$CC?$CFs?$CC@ 0000000180003a00     libmexit01.obj
 0002:00000a20       ??_C@_0BC@IDKJNIMD@?0?5expected?3?5?$CC?$CFs?$CC?6@ 0000000180003a20     libmexit01.obj
 0002:00000a38       ??_C@_0CE@IJAEBHNF@?$CIexit?$CD?$CFllu?$CJ?5wrong?5method?5name?3?5@ 0000000180003a38     libmexit01.obj
 0002:00000a60       ??_C@_0CD@KBECCNJI@?$CIexit?$CD?$CFllu?$CJ?5wrong?5method?5sig?3?5?$CC@ 0000000180003a60     libmexit01.obj
 0002:00000a88       ??_C@_0BP@GPEOAICM@?$CIexit?$CD?$CFllu?$CJ?5wrong?5location?3?5?$CFs@ 0000000180003a88     libmexit01.obj
 0002:00000aa8       ??_C@_0BA@OJCFFGGB@?0?5expected?3?5?$CFs?6@ 0000000180003aa8     libmexit01.obj
 0002:00000ab8       ??_C@_0DJ@NPAECGPK@The?5thread?5IsVirtualThread?5?$CFd?5d@ 0000000180003ab8     libmexit01.obj
 0002:00000af8       ??_C@_0CA@BGJIKHIC@Unexpected?5method?5exit?5catched?3@ 0000000180003af8     libmexit01.obj
 0002:00000b18       ??_C@_0BC@ECKNJPDP@?5?5?5?5?5class?3?5?$CC?$CFs?$CC?6@ 0000000180003b18     libmexit01.obj
 0002:00000b30       ??_C@_0BE@EDAJGJA@?5?5?5?5method?3?5?$CC?$CFs?$CFs?$CC?6@ 0000000180003b30     libmexit01.obj
 0002:00000b48       ??_C@_0BA@EPDHOKNE@?5?5location?3?5?$CFs?6@ 0000000180003b48     libmexit01.obj
 0002:00000b58       ??_C@_0CJ@KCDEKOCJ@Wrong?5result?5of?5a?5valid?5call?5to@ 0000000180003b58     libmexit01.obj
 0002:00000b88       ??_C@_0DG@LAJPGIIE@?$CIGetPotentialCapabilities?$CJ?5unex@ 0000000180003b88     libmexit01.obj
 0002:00000bc0       ??_C@_0CN@LKPEOJPO@?$CIAddCapabilities?$CJ?5unexpected?5er@ 0000000180003bc0     libmexit01.obj
 0002:00000bf0       ??_C@_0CN@BCCBOHCH@?$CIGetCapabilities?$CJ?5unexpected?5er@ 0000000180003bf0     libmexit01.obj
 0002:00000c20       ??_C@_0CP@IMINGNLL@?$CISetEventCallbacks?$CJ?5unexpected?5@ 0000000180003c20     libmexit01.obj
 0002:00000c50       ??_C@_0CO@DJHOJGID@Warning?3?5MethodExit?5event?5is?5no@ 0000000180003c50     libmexit01.obj
 0002:00000c80       ??_C@_0CH@CDOJMNAO@JVMTI?5client?5was?5not?5properly?5l@ 0000000180003c80     libmexit01.obj
 0002:00000ca8       ??_C@_0DJ@OMMCJEPI@Failed?5to?5enable?5JVMTI_EVENT_ME@ 0000000180003ca8     libmexit01.obj
 0002:00000ce8       ??_C@_0CH@LPNKMHEN@Failed?5to?5get?5current?5thread?3?5?$CF@ 0000000180003ce8     libmexit01.obj
 0002:00000d10       ??_C@_08HJJLIIEM@mexit01a@ 0000000180003d10     libmexit01.obj
 0002:00000d20       ??_C@_0CI@ENGKOKKF@Cannot?5find?5MethodExit?4mexit01a@ 0000000180003d20     libmexit01.obj
 0002:00000d48       ??_C@_0BO@OPCEIILC@Cannot?5find?5metod?5?$CCdummy?$CI?$CJ?$CC?$CB?6@ 0000000180003d48     libmexit01.obj
 0002:00000d68       ??_C@_0DK@ONFPOBAG@Failed?5to?5disable?5JVMTI_EVENT_M@ 0000000180003d68     libmexit01.obj
 0002:00000da8       ??_C@_0DJ@FFHEPCJP@Wrong?5number?5of?5MethodExit?5even@ 0000000180003da8     libmexit01.obj
 0002:00000de8       ??_C@_0BD@ENAMJMLH@Executing?5chain?$CI?$CJ?6@ 0000000180003de8     libmexit01.obj
 0002:00000e00       ??_C@_1EC@JIJBPKFM@?$AAa?$AAp?$AAi?$AA?9?$AAm?$AAs?$AA?9?$AAw?$AAi?$AAn?$AA?9?$AAc?$AAo?$AAr?$AAe@ 0000000180003e00     MSVCRT:thread_safe_statics.obj
 0002:00000e48       ??_C@_1BK@MGMFAEKH@?$AAk?$AAe?$AAr?$AAn?$AAe?$AAl?$AA3?$AA2?$AA?4?$AAd?$AAl?$AAl@ 0000000180003e48     MSVCRT:thread_safe_statics.obj
 0002:00000e68       ??_C@_0BJ@JEBJOJFJ@SleepConditionVariableCS@ 0000000180003e68     MSVCRT:thread_safe_statics.obj
 0002:00000e88       ??_C@_0BJ@PGPPEPCC@WakeAllConditionVariable@ 0000000180003e88     MSVCRT:thread_safe_statics.obj
 0002:00000ea8       _pDefaultRawDllMain        0000000180003ea8     MSVCRT:dll_dllmain.obj
 0002:00000ea8       _pRawDllMain               0000000180003ea8     MSVCRT:dll_dllmain.obj
 0002:00000eb0       __xmm@ffffffffffffffffffffffffffffffff 0000000180003eb0     MSVCRT:utility.obj
 0002:00000ed0       _load_config_used          0000000180003ed0     MSVCRT:loadcfg.obj
 0002:00001080       _tls_used                  0000000180004080     MSVCRT:tlssup.obj
 0002:000010a8       __volatile_metadata        00000001800040a8     <linker-defined>
 0002:00001420       __rtc_iaa                  0000000180004420     MSVCRT:initsect.obj
 0002:00001428       __rtc_izz                  0000000180004428     MSVCRT:initsect.obj
 0002:00001430       __rtc_taa                  0000000180004430     MSVCRT:initsect.obj
 0002:00001438       __rtc_tzz                  0000000180004438     MSVCRT:initsect.obj
 0002:00001440       _tls_start                 0000000180004440     MSVCRT:tlssup.obj
 0002:00001444       _Init_thread_epoch         0000000180004444     MSVCRT:thread_safe_statics.obj
 0002:00001448       _tls_end                   0000000180004448     MSVCRT:tlssup.obj
 0002:000016fc       __IMPORT_DESCRIPTOR_KERNEL32 00000001800046fc     kernel32:KERNEL32.dll
 0002:00001710       __IMPORT_DESCRIPTOR_VCRUNTIME140 0000000180004710     vcruntime:VCRUNTIME140.dll
 0002:00001724       __IMPORT_DESCRIPTOR_api-ms-win-crt-stdio-l1-1-0 0000000180004724     ucrt:api-ms-win-crt-stdio-l1-1-0.dll
 0002:00001738       __IMPORT_DESCRIPTOR_api-ms-win-crt-string-l1-1-0 0000000180004738     ucrt:api-ms-win-crt-string-l1-1-0.dll
 0002:0000174c       __IMPORT_DESCRIPTOR_api-ms-win-crt-runtime-l1-1-0 000000018000474c     ucrt:api-ms-win-crt-runtime-l1-1-0.dll
 0002:00001760       __NULL_IMPORT_DESCRIPTOR   0000000180004760     kernel32:KERNEL32.dll
 0003:00000040       _Init_global_epoch         0000000180005040     MSVCRT:thread_safe_statics.obj
 0003:00000050       __security_cookie          0000000180005050     MSVCRT:gs_cookie.obj
 0003:00000058       __security_cookie_complement 0000000180005058     MSVCRT:gs_cookie.obj
 0003:00000060       __scrt_native_dllmain_reason 0000000180005060     MSVCRT:utility.obj
 0003:00000068       __isa_available            0000000180005068     MSVCRT:cpu_disp.obj
 0003:0000006c       __isa_enabled              000000018000506c     MSVCRT:cpu_disp.obj
 0003:00000070       __memset_fast_string_threshold 0000000180005070     MSVCRT:cpu_disp.obj
 0003:00000078       __memset_nt_threshold      0000000180005078     MSVCRT:cpu_disp.obj
 0003:00000080       __scrt_ucrt_dll_is_in_use  0000000180005080     MSVCRT:ucrt_stubs.obj
 0003:00000090       ?_OptionsStorage@?1??__local_stdio_printf_options@@9@4_KA 0000000180005090     libmexit01.obj
 0003:00000240       _tls_index                 0000000180005240     MSVCRT:tlssup.obj
 0003:00000248       __scrt_current_native_startup_state 0000000180005248     MSVCRT:utility.obj
 0003:00000250       __scrt_native_startup_lock 0000000180005250     MSVCRT:utility.obj
 0003:00000290       __scrt_debugger_hook_flag  0000000180005290     MSVCRT:utility_desktop.obj
 0003:00000810       ?__type_info_root_node@@3U__type_info_node@@A 0000000180005810     MSVCRT:tncleanup.obj
 0003:00000820       ?_OptionsStorage@?1??__local_stdio_scanf_options@@9@4_KA 0000000180005820     MSVCRT:default_local_stdio_options.obj
 0003:00000828       __favor                    0000000180005828     MSVCRT:cpu_disp.obj
 0003:00000830       __dyn_tls_init_callback    0000000180005830     <common>

 entry point at        0001:000011f0

 Static symbols

 0000:ffff8000       .debug$S                   0000000180000000     mexit01.exp
 0000:ffff8000       .debug$S                   0000000180000000     vcruntime:VCRUNTIME140.dll
 0000:ffff8000       .debug$S                   0000000180000000     vcruntime:VCRUNTIME140.dll
 0000:ffff8000       .debug$S                   0000000180000000     vcruntime:VCRUNTIME140.dll
 0000:ffff8000       .debug$S                   0000000180000000     vcruntime:VCRUNTIME140.dll
 0000:ffff8000       .debug$S                   0000000180000000     vcruntime:VCRUNTIME140.dll
 0000:ffff8000       .debug$S                   0000000180000000     vcruntime:VCRUNTIME140.dll
 0000:ffff8000       .debug$S                   0000000180000000     ucrt:api-ms-win-crt-runtime-l1-1-0.dll
 0000:ffff8000       .debug$S                   0000000180000000     ucrt:api-ms-win-crt-runtime-l1-1-0.dll
 0000:ffff8000       .debug$S                   0000000180000000     ucrt:api-ms-win-crt-runtime-l1-1-0.dll
 0000:ffff8000       .debug$S                   0000000180000000     ucrt:api-ms-win-crt-runtime-l1-1-0.dll
 0000:ffff8000       .debug$S                   0000000180000000     ucrt:api-ms-win-crt-runtime-l1-1-0.dll
 0000:ffff8000       .debug$S                   0000000180000000     ucrt:api-ms-win-crt-runtime-l1-1-0.dll
 0000:ffff8000       .debug$S                   0000000180000000     ucrt:api-ms-win-crt-runtime-l1-1-0.dll
 0000:ffff8000       .debug$S                   0000000180000000     ucrt:api-ms-win-crt-runtime-l1-1-0.dll
 0000:ffff8000       .debug$S                   0000000180000000     ucrt:api-ms-win-crt-runtime-l1-1-0.dll
 0000:ffff8000       .debug$S                   0000000180000000     ucrt:api-ms-win-crt-runtime-l1-1-0.dll
 0000:ffff8000       .debug$S                   0000000180000000     ucrt:api-ms-win-crt-runtime-l1-1-0.dll
 0000:ffff8000       .debug$S                   0000000180000000     ucrt:api-ms-win-crt-runtime-l1-1-0.dll
 0000:ffff8000       .debug$S                   0000000180000000     ucrt:api-ms-win-crt-stdio-l1-1-0.dll
 0000:ffff8000       .debug$S                   0000000180000000     ucrt:api-ms-win-crt-stdio-l1-1-0.dll
 0000:ffff8000       .debug$S                   0000000180000000     ucrt:api-ms-win-crt-stdio-l1-1-0.dll
 0000:ffff8000       .debug$S                   0000000180000000     ucrt:api-ms-win-crt-string-l1-1-0.dll
 0000:ffff8000       .debug$S                   0000000180000000     ucrt:api-ms-win-crt-string-l1-1-0.dll
 0000:ffff8000       .debug$S                   0000000180000000     ucrt:api-ms-win-crt-string-l1-1-0.dll
 0000:ffff8000       .debug$S                   0000000180000000     ucrt:api-ms-win-crt-string-l1-1-0.dll
 0000:ffff8000       .debug$S                   0000000180000000     kernel32:KERNEL32.dll
 0000:ffff8000       .debug$S                   0000000180000000     kernel32:KERNEL32.dll
 0000:ffff8000       .debug$S                   0000000180000000     kernel32:KERNEL32.dll
 0000:ffff8000       .debug$S                   0000000180000000     kernel32:KERNEL32.dll
 0000:ffff8000       .debug$S                   0000000180000000     kernel32:KERNEL32.dll
 0000:ffff8000       .debug$S                   0000000180000000     kernel32:KERNEL32.dll
 0000:ffff8000       .debug$S                   0000000180000000     kernel32:KERNEL32.dll
 0000:ffff8000       .debug$S                   0000000180000000     kernel32:KERNEL32.dll
 0000:ffff8000       .debug$S                   0000000180000000     kernel32:KERNEL32.dll
 0000:ffff8000       .debug$S                   0000000180000000     kernel32:KERNEL32.dll
 0000:ffff8000       .debug$S                   0000000180000000     kernel32:KERNEL32.dll
 0000:ffff8000       .debug$S                   0000000180000000     kernel32:KERNEL32.dll
 0000:ffff8000       .debug$S                   0000000180000000     kernel32:KERNEL32.dll
 0000:ffff8000       .debug$S                   0000000180000000     kernel32:KERNEL32.dll
 0000:ffff8000       .debug$S                   0000000180000000     kernel32:KERNEL32.dll
 0000:ffff8000       .debug$S                   0000000180000000     kernel32:KERNEL32.dll
 0000:ffff8000       .debug$S                   0000000180000000     kernel32:KERNEL32.dll
 0000:ffff8000       .debug$S                   0000000180000000     kernel32:KERNEL32.dll
 0000:ffff8000       .debug$S                   0000000180000000     kernel32:KERNEL32.dll
 0000:ffff8000       .debug$S                   0000000180000000     kernel32:KERNEL32.dll
 0000:ffff8000       .debug$S                   0000000180000000     kernel32:KERNEL32.dll
 0000:ffff8000       .debug$S                   0000000180000000     kernel32:KERNEL32.dll
 0000:ffff8000       .debug$S                   0000000180000000     kernel32:KERNEL32.dll
 0000:ffff8000       .debug$S                   0000000180000000     kernel32:KERNEL32.dll
 0000:ffff8000       .debug$S                   0000000180000000     kernel32:KERNEL32.dll
 0000:ffff8000       .debug$S                   0000000180000000     kernel32:KERNEL32.dll
 0000:ffff8000       .debug$S                   0000000180000000     kernel32:KERNEL32.dll
 0000:ffff8000       .debug$S                   0000000180000000     kernel32:KERNEL32.dll
 0001:00000d24       ?__scrt_initialize_thread_safe_statics@@YAHXZ 0000000180001d24 f   MSVCRT:thread_safe_statics.obj
 0001:00000df4       ?__scrt_uninitialize_thread_safe_statics@@YAXXZ 0000000180001df4 f   MSVCRT:thread_safe_statics.obj
 0001:00000ea0       $$000000                   0000000180001ea0     MSVCRT:amdsecgs.obj
 0001:00000ed0       ?dllmain_crt_dispatch@@YAHQEAUHINSTANCE__@@KQEAX@Z 0000000180001ed0 f   MSVCRT:dll_dllmain.obj
 0001:00000f20       ?dllmain_crt_process_attach@@YAHQEAUHINSTANCE__@@QEAX@Z 0000000180001f20 f   MSVCRT:dll_dllmain.obj
 0001:00001038       ?dllmain_crt_process_detach@@YAH_N@Z 0000000180002038 f   MSVCRT:dll_dllmain.obj
 0001:000010bc       ?dllmain_dispatch@@YAHQEAUHINSTANCE__@@KQEAX@Z 00000001800020bc f   MSVCRT:dll_dllmain.obj
 0001:00001810       capture_previous_context   0000000180002810 f   MSVCRT:gs_report.obj
 0001:00001c50       $$000000                   0000000180002c50     MSVCRT:guard_dispatch.obj
 0001:00001c70       $$000000                   0000000180002c70     MSVCRT:guard_xfg_dispatch.obj
 0001:00001c86       ?fin$0@?0??dllmain_crt_process_attach@@YAHQEAUHINSTANCE__@@QEAX@Z@4HA 0000000180002c86 f   MSVCRT:dll_dllmain.obj
 0001:00001c9d       ?fin$0@?0??dllmain_crt_process_detach@@YAH_N@Z@4HA 0000000180002c9d f   MSVCRT:dll_dllmain.obj
 0001:00001cb6       ?fin$1@?0??dllmain_crt_process_detach@@YAH_N@Z@4HA 0000000180002cb6 f   MSVCRT:dll_dllmain.obj
 0001:00001cca       ?filt$0@?0??dllmain_dispatch@@YAHQEAUHINSTANCE__@@KQEAX@Z@4HA 0000000180002cca f   MSVCRT:dll_dllmain.obj
 0001:00001d00       __scrt_is_nonwritable_in_current_image$filt$0 0000000180002d00 f   MSVCRT:utility.obj
 0002:000001b0       ?__scrt_initialize_tss_var@@3P6AHXZEA 00000001800031b0     MSVCRT:thread_safe_statics.obj
 0002:00000ec0       GS_ExceptionPointers       0000000180003ec0     MSVCRT:gs_report.obj
 0002:00001450       $unwind$printf             0000000180004450     libmexit01.obj
 0002:0000145c       $unwind$?CallStaticVoidMethod@JNIEnv_@@QEAAXPEAV_jclass@@PEAU_jmethodID@@ZZ 000000018000445c     libmexit01.obj
 0002:00001464       $unwind$?jlong_to_string@@YAPEAD_JPEAD@Z 0000000180004464     libmexit01.obj
 0002:00001474       $unwind$MethodExit         0000000180004474     libmexit01.obj
 0002:00001490       $unwind$Agent_Initialize   0000000180004490     libmexit01.obj
 0002:000014a0       $unwind$Java_mexit01_init0 00000001800044a0     libmexit01.obj
 0002:000014a0       $unwind$__raise_securityfailure 00000001800044a0     MSVCRT:gs_report.obj
 0002:000014a0       $unwind$__scrt_initialize_crt 00000001800044a0     MSVCRT:utility.obj
 0002:000014a0       $unwind$__scrt_initialize_onexit_tables 00000001800044a0     MSVCRT:utility.obj
 0002:000014a0       $unwind$__scrt_release_startup_lock 00000001800044a0     MSVCRT:utility.obj
 0002:000014a0       $unwind$__scrt_uninitialize_crt 00000001800044a0     MSVCRT:utility.obj
 0002:000014a0       $unwind$_onexit            00000001800044a0     MSVCRT:utility.obj
 0002:000014a8       $unwind$Java_mexit01_check 00000001800044a8     libmexit01.obj
 0002:000014b4       $unwind$Java_mexit01a_chain 00000001800044b4     libmexit01.obj
 0002:000014b4       $unwind$__scrt_initialize_default_local_stdio_options 00000001800044b4     MSVCRT:default_local_stdio_options.obj
 0002:000014b4       $unwind$?dllmain_crt_dispatch@@YAHQEAUHINSTANCE__@@KQEAX@Z 00000001800044b4     MSVCRT:dll_dllmain.obj
 0002:000014b4       $unwind$DllMain            00000001800044b4     MSVCRT:dll_dllmain_stub.obj
 0002:000014b4       $unwind$__GSHandlerCheck   00000001800044b4     MSVCRT:gshandler.obj
 0002:000014b4       $unwind$?__scrt_uninitialize_thread_safe_statics@@YAXXZ 00000001800044b4     MSVCRT:thread_safe_statics.obj
 0002:000014b4       $unwind$__scrt_acquire_startup_lock 00000001800044b4     MSVCRT:utility.obj
 0002:000014b4       $unwind$__scrt_dllmain_after_initialize_c 00000001800044b4     MSVCRT:utility.obj
 0002:000014b4       $unwind$__scrt_dllmain_before_initialize_c 00000001800044b4     MSVCRT:utility.obj
 0002:000014b4       $unwind$__scrt_dllmain_crt_thread_attach 00000001800044b4     MSVCRT:utility.obj
 0002:000014b4       $unwind$__scrt_dllmain_crt_thread_detach 00000001800044b4     MSVCRT:utility.obj
 0002:000014b4       $unwind$__scrt_dllmain_uninitialize_c 00000001800044b4     MSVCRT:utility.obj
 0002:000014b4       $unwind$__scrt_dllmain_uninitialize_critical 00000001800044b4     MSVCRT:utility.obj
 0002:000014b4       $unwind$atexit             00000001800044b4     MSVCRT:utility.obj
 0002:000014bc       $unwind$_RTC_Initialize    00000001800044bc     MSVCRT:initsect.obj
 0002:000014bc       $unwind$_RTC_Terminate     00000001800044bc     MSVCRT:initsect.obj
 0002:000014bc       $unwind$?__scrt_initialize_thread_safe_statics@@YAHXZ 00000001800044bc     MSVCRT:thread_safe_statics.obj
 0002:000014c8       $unwind$__GSHandlerCheckCommon 00000001800044c8     MSVCRT:gshandler.obj
 0002:000014d0       $xdatasym                  00000001800044d0     MSVCRT:amdsecgs.obj
 0002:000014d4       $unwind$?dllmain_crt_process_attach@@YAHQEAUHINSTANCE__@@QEAX@Z 00000001800044d4     MSVCRT:dll_dllmain.obj
 0002:00001510       $unwind$?fin$0@?0??dllmain_crt_process_attach@@YAHQEAUHINSTANCE__@@QEAX@Z@4HA 0000000180004510     MSVCRT:dll_dllmain.obj
 0002:00001510       $unwind$?fin$0@?0??dllmain_crt_process_detach@@YAH_N@Z@4HA 0000000180004510     MSVCRT:dll_dllmain.obj
 0002:00001510       $unwind$?fin$1@?0??dllmain_crt_process_detach@@YAH_N@Z@4HA 0000000180004510     MSVCRT:dll_dllmain.obj
 0002:00001518       $unwind$?dllmain_crt_process_detach@@YAH_N@Z 0000000180004518     MSVCRT:dll_dllmain.obj
 0002:0000156c       $unwind$?dllmain_dispatch@@YAHQEAUHINSTANCE__@@KQEAX@Z 000000018000456c     MSVCRT:dll_dllmain.obj
 0002:00001594       $unwind$?filt$0@?0??dllmain_dispatch@@YAHQEAUHINSTANCE__@@KQEAX@Z@4HA 0000000180004594     MSVCRT:dll_dllmain.obj
 0002:0000159c       $unwind$_DllMainCRTStartup 000000018000459c     MSVCRT:dll_dllmain.obj
 0002:000015ac       $unwind$__scrt_is_nonwritable_in_current_image 00000001800045ac     MSVCRT:utility.obj
 0002:000015cc       $unwind$__scrt_is_nonwritable_in_current_image$filt$0 00000001800045cc     MSVCRT:utility.obj
 0002:000015d4       $unwind$__scrt_dllmain_exception_filter 00000001800045d4     MSVCRT:utility.obj
 0002:000015e8       $unwind$__scrt_fastfail    00000001800045e8     MSVCRT:utility_desktop.obj
 0002:000015f8       $unwind$__report_gsfailure 00000001800045f8     MSVCRT:gs_report.obj
 0002:00001600       $unwind$capture_previous_context 0000000180004600     MSVCRT:gs_report.obj
 0002:0000160c       $unwind$__security_init_cookie 000000018000460c     MSVCRT:gs_support.obj
 0002:00001618       $unwind$__isa_available_init 0000000180004618     MSVCRT:cpu_disp.obj
 0002:00001628       $xdatasym                  0000000180004628     MSVCRT:guard_dispatch.obj
 0002:00001630       $xdatasym                  0000000180004630     MSVCRT:guard_xfg_dispatch.obj
 0002:00001640       .edata                     0000000180004640     mexit01.exp
 0002:00001668       rgpv                       0000000180004668     mexit01.exp
 0002:0000167c       rgszName                   000000018000467c     mexit01.exp
 0002:00001690       rgwOrd                     0000000180004690     mexit01.exp
 0002:0000169a       szName                     000000018000469a     mexit01.exp
 0002:000016a6       $N00001                    00000001800046a6     mexit01.exp
 0002:000016b5       $N00002                    00000001800046b5     mexit01.exp
 0002:000016c2       $N00003                    00000001800046c2     mexit01.exp
 0002:000016d5       $N00004                    00000001800046d5     mexit01.exp
 0002:000016e8       $N00005                    00000001800046e8     mexit01.exp
 0002:00001ac2       .idata$6                   0000000180004ac2     kernel32:KERNEL32.dll
 0002:00001b12       .idata$6                   0000000180004b12     vcruntime:VCRUNTIME140.dll
 0002:00001c34       .idata$6                   0000000180004c34     ucrt:api-ms-win-crt-stdio-l1-1-0.dll
 0002:00001c54       .idata$6                   0000000180004c54     ucrt:api-ms-win-crt-string-l1-1-0.dll
 0002:00001c76       .idata$6                   0000000180004c76     ucrt:api-ms-win-crt-runtime-l1-1-0.dll
 0003:00000000       exits                      0000000180005000     libmexit01.obj
 0003:000000a0       jvmti                      00000001800050a0     libmexit01.obj
 0003:000000a8       result                     00000001800050a8     libmexit01.obj
 0003:000000ac       isVirtualExpected          00000001800050ac     libmexit01.obj
 0003:000000b0       callbacks                  00000001800050b0     libmexit01.obj
 0003:000001e8       eventsExpected             00000001800051e8     libmexit01.obj
 0003:000001f0       eventsCount                00000001800051f0     libmexit01.obj
 0003:000001f8       ?g_tss_cv@@3U_RTL_CONDITION_VARIABLE@@A 00000001800051f8     MSVCRT:thread_safe_statics.obj
 0003:00000200       ?g_tss_event@@3PEAXEA      0000000180005200     MSVCRT:thread_safe_statics.obj
 0003:00000208       ?g_tss_mutex@@3U_RTL_CRITICAL_SECTION@@A 0000000180005208     MSVCRT:thread_safe_statics.obj
 0003:00000230       ?g_sleep_condition_variable_cs@@3P6AHPEAU_RTL_CONDITION_VARIABLE@@PEAU_RTL_CRITICAL_SECTION@@K@ZEA 0000000180005230     MSVCRT:thread_safe_statics.obj
 0003:00000238       ?g_wake_all_condition_variable@@3P6AXPEAU_RTL_CONDITION_VARIABLE@@@ZEA 0000000180005238     MSVCRT:thread_safe_statics.obj
 0003:00000244       ?__proc_attached@@3HA      0000000180005244     MSVCRT:dll_dllmain.obj
 0003:00000258       ?is_initialized_as_dll@@3_NA 0000000180005258     MSVCRT:utility.obj
 0003:00000259       ?module_local_atexit_table_initialized@@3_NA 0000000180005259     MSVCRT:utility.obj
 0003:00000260       ?module_local_atexit_table@@3U_onexit_table_t@@A 0000000180005260     MSVCRT:utility.obj
 0003:00000278       ?module_local_at_quick_exit_table@@3U_onexit_table_t@@A 0000000180005278     MSVCRT:utility.obj
 0003:000002a0       GS_ExceptionRecord         00000001800052a0     MSVCRT:gs_report.obj
 0003:00000340       GS_ContextRecord           0000000180005340     MSVCRT:gs_report.obj
